:100000000C9476010C94AE010C94AE010C94AE01EC
:100010000C94AE010C94AE010C94AE010C94AE01A4
:100020000C94AE010C94AE010C94980E0C94D40D6B
:100030000C94CF150C94AE010C94AE010C94AE014F
:100040000C94AE010C94AE010C94AE010C94AE0174
:100050000C94AE010C94930F0C94AE010C94AE0171
:100060000C94AE010C94AE010C94AE010C94AE0154
:100070000C94AE010C94AE010C94AE010C94AE0144
:100080000C94AE010C94AE010C94AE010C94AE0134
:100090000C94AE010C94AE010C94AE010C94AE0124
:1000A0000C94AE010C94AE010C94AE01D306D306B1
:1000B0000507050777071F091F091F09930771081F
:1000C00082088208ED0B140CAC0D140CAC0D5C0C0A
:1000D0007F0CAC0D6E0D810D05010980A10185031A
:1000E00019012AB700150126B70095017510810086
:1000F000C0050C0901A101850419012AA0021501FE
:1001000026A002950175108100C005010906A10114
:10011000050719E029E715002501950875018102F9
:100120009501750881010507190029FF150026FFB3
:1001300000950675088100050819012905950575C2
:10014000019102950175039101C009023B00020172
:1001500000A0FA09040000010301010009211101B6
:100160000001224000070581030800010904010085
:1001700001030000000921110100012232000705DE
:100180008203200001120100020000000857530101
:1001900000010001020001120344007900730074A1
:1001A000006F0070006900610000002203530061CD
:1001B000006E0063007400690066006900650064F9
:1001C000002E0057006F0072006B007300000004E7
:1001D00003090429001E002000210022002300241E
:1001E000002500260027002D002E00350031002BB1
:1001F000001F001A000800150017001C0018000C52
:1002000000120013002F0030002A003900140016DD
:1002100000070009000A000B000D000E000F00335C
:1002200000340028004C00E10004001B0006001907
:1002300000050005001100360037003800E50052C7
:10024000004B00E0001D00E20000002C0001512CDA
:10025000001000E600E400500051004F004E003551
:10026000003A003C003D003E003F0040004100429B
:10027000004300440045000100010001003B000173
:100280000001000100010001000100010001000166
:100290000001000100010001000100010001000156
:1002A0000001000100010001000100010001000146
:1002B00000490001000100010001000100010001EE
:1002C000000100010001000100010001004A00E3FB
:1002D0000001000100000001000100010001000117
:1002E0000001000100010001004D000011241FBEAB
:1002F000CFEFDAE0DEBFCDBF04B603FE18C08091B9
:10030000230290912402A0912502B0912602873009
:10031000904BA740B04B59F4109223021092240244
:100320001092250210922602E0E0F8E3099511E010
:10033000A0E0B1E0EAEAF1E302C005900D92A23537
:10034000B107D9F722E0A2E5B1E001C01D92A332C6
:10035000B207E1F70E94E0160C94D3180C94000049
:100360002EE0929F800D1124682F66956695669504
:10037000982F977085E0689FB001112440E050E00D
:1003800080E0FB01E40FF51FEB5AFE4F208130E0C7
:10039000092E02C0369527950A94E2F7217033277B
:1003A000042E01C0220F0A94EAF7822B4F5F5F4FA1
:1003B0004530510531F708952EE0929F800D1124AC
:1003C000E82FE695E695E695877051E001C0550F58
:1003D0008A95EAF785E0E89FF0011124EB5AFE4F79
:1003E00020E030E070E04081CB01022E02C0969503
:1003F00087950A94E2F78170819584278523842765
:1004000081932F5F3F4F2530310569F7089580E0D4
:1004100090E00E94281680E090E00E941216109250
:10042000E9010C9426136093FD017093FE01809303
:10043000FF01909300020C9407020F931F9341E079
:1004400050E060E070E004C0440F551F661F771F46
:100450008A95D2F78091FD019091FE01A091FF0154
:10046000B09100028A019B01082B192B2A2B3B2BF0
:10047000C901B8011F910F910C9413028F929F92A2
:10048000AF92BF92DF92EF92FF920F931F93CF93A1
:10049000DF938090FD019090FE01A090FF01B0904D
:1004A00000024091EC015091ED016091EE017091DC
:1004B000EF01842A952AA62AB72ACFE1D0E02EE0C0
:1004C000929F7001112496E4D92E082F10E0D501D7
:1004D000C4010C2E04C0B695A795979587950A94EC
:1004E000D2F780FD04C0219790F780E014C0DC9E15
:1004F000F001DD9EF00D1124EE0DFF1DE00FF11F48
:10050000EE0FFF1FED52FE4F859194910E94141142
:10051000019749F38C2FDF91CF911F910F91FF909D
:10052000EF90DF90BF90AF909F908F9008950F93C2
:100530001F9341E050E060E070E004C0440F551F9D
:10054000661F771F8A95D2F74095509560957095F4
:100550008091FD019091FE01A091FF01B0910002F8
:100560008A019B01082319232A233B23C901B801CF
:100570001F910F910C9413026093EC017093ED01A5
:100580008093EE019093EF010C940702FC018081AF
:1005900091810E94121492959F70963079F010F418
:1005A000925001C09A50923068F4803F69F018F47C
:1005B000883E40F409C0843F29F406C0883E20F0FC
:1005C000813F11F080E0089581E008951092EA01E2
:1005D00086E0E2EAF1E0DF011D928A95E9F70C94EA
:1005E0000702882321F00E941F130C9426130895FC
:1005F000882339F09091EA01892B8093EA010C94C9
:1006000026130895882371F19CEF980F913A60F4B6
:10061000E0EAF1E09281891301C01282319691E003
:10062000E63AF907B9F70DC090E2980F983058F400
:10063000982F977081E001C0880F9A95EAF70E9481
:100640001F130C9426139BE5980F933020F480E041
:1006500090E00C942816885A873120F480E090E0CE
:100660000C9412160895CF93882309F453C09CEF7D
:10067000980F913AF8F4C82FE2EAF1E088EA91E0A5
:100680002191C21721F08E179F07D1F70DC0E0EA24
:10069000F1E08281C81301C01282319641E0E63A4E
:1006A000F407B9F70E9426136C2F80EA91E00E94AC
:1006B000F81513C090E2980F983090F4877021E0FD
:1006C00030E0A90102C0440F551F8A95E2F7CA0124
:1006D0009091EA01892B8093EA01CF910C94261323
:1006E000EBE5E80FE33040F4F0E0E35FFE4F80819C
:1006F00090E0CF910C942816885A873158F4E82F4F
:10070000F0E0EE0FFF1FE05FFE4F80819181CF91FF
:100710000C941216CF9108951F93CF93DF93CDB70A
:10072000DEB767970FB6F894DEBF0FBECDBF4B8B19
:100730005C8B6D8B7E8B8F8B61111092E90186E053
:100740009E01235F3F4FD901E82F1D92EA95E9F7FB
:1007500095E0FE017396D90101900D929A95E1F70B
:100760009C894E895F897B897D879E876F87598B9E
:10077000488BF901DE01179601900D928A95E1F7F9
:10078000CE0107960E942E1481113EC086E0FE0124
:100790003796DE01119601900D928A95E1F7FF815F
:1007A000E8856A857B856115710531F0EF3F31F48D
:1007B00081E0FF3F19F403C081E001C080E080FDCB
:1007C00023C02091AE0130E0C901019687709927BE
:1007D0004091DF0150E08417950779F1F983EA83AE
:1007E0007D836C8396E0929FD001939FB00D11247E
:1007F000A155BE4FFE01319601900D929A95E1F7F9
:100800008093AE010E949C1316E08091DF019091CD
:10081000AE018917F9F0189FC001112481559E4F30
:100820000E942E148823B1F08091DF0190E00196A0
:10083000877099278093DF01E8CF0E94E60210922B
:10084000AE011092DF01E8EAF1E086E0DF011D92DF
:100850008A95E9F767960FB6F894DEBF0FBECDBF55
:10086000DF91CF911F9108958F929F92AF92BF9287
:10087000CF92DF92EF92FF920F931F93CF93DF936C
:10088000CDB7DEB72A970FB6F894DEBF0FBECDBF47
:10089000FC010081D18083819481892B39F01FEF85
:1008A000D11206C091E00F3F19F403C091E001C0DE
:1008B00090E090FD24C57F0185E0DE011696019051
:1008C0000D928A95E1F7F70122818E819F81222383
:1008D00049F00E943E02182F682F8E819F810E944E
:1008E000DC0103C00E94B001182F26E4129FF00122
:1008F00011243EE0D39EE00DF11D1124E00FF11D07
:10090000EE0FFF1FED52FE4F05911491043F8CE551
:10091000180741F190F4093DECE51E07E9F00A3DA6
:10092000FCE51F0789F1083D2CE51207B1F506E249
:1009300021EE41EE68ED7CE52CC0063F3CE5130757
:10094000E9F0B0F0073F9CE5190739F507E225EE1D
:1009500046EE67EF7CE51DC007E225EE45EE69ED4A
:100960007CE517C006E221EE40EE64EF7CE511C0A5
:1009700007E225EE44EE65EF7CE50BC006E221EED2
:1009800042EE66EF7CE505C008E221E045EE6AED47
:100990007CE5C7010E944A168FC4F7018281882333
:1009A00009F45BC110921B020430FDE51F0758F4E7
:1009B0000B3F2CE5120780F4C80182509C454497F8
:1009C00008F035C109C002363DE5130729F0063AA3
:1009D0008DE5180709F02BC10E949D129093020229
:1009E0008093010201319CE5190709F4C6C008F0A3
:1009F00042C00930FCE51F0709F49BC000F5053033
:100A00003CE5130709F485C078F403309CE5190729
:100A100009F478C008F07AC002301C4509F0F7C02C
:100A2000809101028160F1C007302CE5120709F4C2
:100A300078C008F07AC0809101028061E6C00D3074
:100A40008CE5180709F487C058F40B30ECE51E0755
:100A500009F479C008F07BC08091010288606FC002
:100A60000F302CE5120709F480C008F082C0809195
:100A70000102877FCAC00E3F8CE5180709F471C0D8
:100A800000F50531ECE51E0709F485C068F4033173
:100A90002CE5120709F475C008F095C00E94E60223
:100AA000809101028F77B1C00C3F8CE51807A9F146
:100AB00008F054C00B3F1C4509F0A9C08091020208
:100AC00040C00230FDE51F0709F489C058F4011544
:100AD0003DE5130709F45AC008F069C0809102028D
:100AE00082602FC002369DE5190709F47EC0063AE0
:100AF000EDE51E0709F483C003301D4509F087C0EA
:100B000060E06EC08091010282607FC0809101022E
:100B100016C080910102886078C0809102028260D4
:100B20004FC080910102806270C080910102806498
:100B30006CC00E94E60280910102806866C08460F9
:100B400064C081603DC0809101028E7F5EC0809153
:100B500001028D7F5AC08091010216C0809102026D
:100B600018C0809102028D7F2BC0809101028F7E80
:100B70004CC0809101028F7D48C0809101028F7B23
:100B800044C080910102877F8B7F3FC08091020229
:100B90008D7F8E7F15C08091010282FB222720F974
:100BA00091E0922790FB82F990FB83F92EC080910F
:100BB0000202982F909591708E7F892B90FB81F97E
:100BC0008093020224C00E94E6028091010287FB0A
:100BD000222720F991E0922790FB87F916C061E067
:100BE0008EE090E00E948C1812C08091010284FB7C
:100BF000222720F991E0922790FB84F906C080918A
:100C00000102982F909590FB80F9809301026091EA
:100C100001021091020284E090E00E948C18612F82
:100C200082E290E00E948C180E94E60245C30631E1
:100C30002CE5120759F58091EA018A7A91E009F4CE
:100C400090E090935401882311F065E301C069E2BC
:100C500080EA91E00E94F81516C006311C4509F0A3
:100C600046C080915401882309F447C385E3E0EA34
:100C7000F1E026EA31E09281891301C012823196B7
:100C80002E173F07C1F70E94261316C30B352DE51B
:100C9000120741F150F401158CE51807A9F00F3D3A
:100CA0001C4529F50E94AE1207C30C35EDE51E0761
:100CB000D9F00D351D45D9F48091020282FB8827B9
:100CC00080F991E0892711C00E94E6020FEF14E33A
:100CD0002CE0015010402040E1F700C000000E94CD
:100CE0006F0FEAC281E001C080E00E947F13F7012C
:100CF00082810081D180882359F0802F9D2D0E9410
:100D00003E02182F682F802F9D2D0E94DC0105C008
:100D1000802F9D2D0E94B001182F26E4129FF00114
:100D200011243EE0D39EE00DF11D1124E00FF11DD2
:100D3000EE0FFF1FED52FE4F859194910E9414110A
:100D40008C01982EF701D280A580A2943FE0A322C7
:100D50008091E0018770B9F0DD20A9F0812F807FBC
:100D6000803421F080E2800F883068F080910202A8
:100D700082FD09C082E00E9462138091E0018770C9
:100D8000CC24C3948111C12CB12EB2949FE0B9221E
:100D90008B2D90E08C30910508F051C2FC01EA5A8D
:100DA000FF4F0C94C018812F807F1F70882311F093
:100DB0001295107FDD20B9F0112309F42DC280E2D5
:100DC000800F883010F0911006C08091EA01182B36
:100DD0001093EA0105C08091E901182B1093E901F5
:100DE0000E94261319C2802F0E940203112309F4C6
:100DF00026C2005E083078F1992069F11095809143
:100E0000E90118231093E90129C0812F807F1F7009
:100E1000803211F01295107F992021F0F1E09F1699
:100E2000D9F149C08091020282FF1BC0DD2069F028
:100E3000112339F08091EA01182B1093EA010E94E6
:100E4000261380E00E943303FAC180E00E9402036F
:100E5000112309F4F4C1812F0E941F130E9426134D
:100E6000EEC1DD2081F08091EB01AA2051F001E07C
:100E7000A01207C0182B181709F4E1C11093EB0159
:100E8000DEC1812B10C0AA2021F021E0A21609F4B6
:100E9000D6C10E94191327C0DD2041F035E03A1574
:100EA00008F4CDC1812F0E94F802C9C184E08A15DF
:100EB00008F4C5C118C0DD2049F0AA2099F3F70154
:100EC000858180FFA9C18F708583ECCFAA2059F05E
:100ED000093309F0B1C1FFEF17EE23E0F1501040E4
:100EE0002040E1F7A7C1812F0E94F102A8C1812F04
:100EF00086958695837019F0813059F0A0C1DD2068
:100F000019F0C801937002C080E090E00E9428169A
:100F10009CC1DD2019F0C801937002C080E090E010
:100F20000E94121692C1812F837009F069C0D110FE
:100F30008AC1902F929596959770990F990F802F4F
:100F40008F70882E912CA12CB12C092E04C0880CF6
:100F5000991CAA1CBB1C0A94D2F704FF12C04FE0D4
:100F600050E060E070E004C0440F551F661F771F1B
:100F70009A95D2F7DB01CA0180959095A095B0951E
:100F800003C080E090E0DC0116951695412F437078
:100F9000423019F1C8F40091EC011091ED0120915B
:100FA000EE013091EF01413059F088299929AA29A1
:100FB000BB29BC01CD0160237123822393230AC086
:100FC000802A912AA22AB32ABC01CD016829792955
:100FD0008A299B290E94BC0236C188299929AA29FD
:100FE000BB290091EC011091ED012091EE013091AF
:100FF000EF01BC01CD016027712782279327EACF3B
:10100000DD2019F0812F817001C08695882309F4B5
:101010001AC1902F929596959770990F990F802FDE
:101020008F70882E912CA12CB12C092E04C0880C15
:10103000991CAA1CBB1C0A94D2F704FF12C04FE0F3
:1010400050E060E070E004C0440F551F661F771F3A
:101050009A95D2F7DB01CA0180959095A095B0953D
:1010600003C080E090E0DC0116951695412F437097
:101070004230D9F068F50091FD011091FE012091F8
:10108000FF0130910002413059F088299929AA299D
:10109000BB29BC01CD0160237123822393231EC091
:1010A000802A912AA22AB32A13C088299929AA2919
:1010B000BB290091FD011091FE012091FF013091AB
:1010C0000002BC01CD01602771278227932706C04B
:1010D000BC01CD01682979298A299B290E94130224
:1010E000B2C01F70DD2039F0812F0E941D02802FB9
:1010F0000E94F802A8C0802F0E94F102812F0E9456
:101100009702A1C0802F32EF931609F443C039151E
:1011100038F090EF991659F0E1EF9E16B1F177C0D3
:10112000F3EF9F16F1F124EF921659F170C0DD2014
:1011300019F134E03A1508F482C01F7181E090E0A3
:10114000A0E0B0E0AC01BD0104C0440F551F661F14
:10115000771F1A95D2F78091FD019091FE01A09121
:10116000FF01B09100028A019B01082719272A2755
:101170003B27C901B80129C025E02A1508F45FC042
:10118000DCCF8091020282FF23C0DD2029F0812F75
:101190008F7130C0DD20D9F3812F8F710E949702AB
:1011A0004EC0DD2079F01F7181E090E0A0E0B0E05A
:1011B000BC01CD0104C0660F771F881F991F1A95C7
:1011C000D2F703C060E070E0CB010E94130237C089
:1011D000DD2099F01F71812F0E941D028091020273
:1011E00082FD07C038E0139FC00111248360809303
:1011F000E001812F0E941D0222C081E00E94621343
:1012000081E08A15E0F482E00E94621318C0DD20BC
:1012100029F0AA2009F4BBCF802F14CEAA2009F40C
:10122000BBCF893349F49FEFE7EEF3E09150E04004
:10123000F040E1F700C00000802F0E94020388EF19
:101240008B0D843010F40E943E16CC20A9F08091C2
:10125000E00180FD11C0F701128285958595859585
:101260000E941D02C7010E9434048091E00185950F
:10127000859585950E94970285E0F701DE0111961C
:1012800001900D928A95E1F789819A810E94B001BF
:101290009A8106E4809FF00111241EE0919FE00DE9
:1012A000F11D11248981E80FF11DEE0FFF1FED5292
:1012B000FE4F8591949123C08091E0018770F9F0F1
:1012C000F70182818823D9F08091020282FD17C044
:1012D00082E02A960FB6F894DEBF0FBECDBFDF9135
:1012E000CF911F910F91FF90EF90DF90CF90BF9023
:1012F000AF909F908F900C94621389E2B8CC2A969D
:101300000FB6F894DEBF0FBECDBFDF91CF911F9116
:101310000F91FF90EF90DF90CF90BF90AF909F9094
:101320008F9008952091E4003091E50095E640917A
:10133000EC00842F817040FF23C08091E80080FD85
:101340001DC080919601882399F0853099F0809195
:10135000EB0085FD11C04091E4005091E500241799
:10136000350729F3915011F09A01E1CF84E00895F7
:1013700082E0089583E0089581E0089580E0089573
:101380004091E80042FFDDCF0895EF92FF920F9366
:101390001F93CF93DF937C018B010E9492098111EF
:1013A00019C0E70101151105A1F08091E80085FD44
:1013B0000AC08091E8008E778093E8000E9492092D
:1013C000882381F307C089918093F10001501109AE
:1013D000E9CF80E0DF91CF911F910F91FF90EF90C7
:1013E00008958091980187FF11C08091E80082FDE7
:1013F00005C0809196018111F8CF11C08091E8005D
:101400008B770BC080919601882349F08091E8008A
:1014100080FFF8CF8091E8008E778093E8000895F0
:10142000982F973068F59093E900981739F07091EC
:10143000EC002091ED005091F00003C0242F762F96
:1014400050E021FD02C09F5FECCF3091EB003E7F6A
:101450003093EB003091ED003D7F3093ED00309103
:10146000EB0031603093EB007093EC002093ED00C3
:101470005093F0002091EE0027FDE5CF80E0089525
:101480008F708093E90081E0089520919E01309152
:101490009F012617370748F06115710539F420912F
:1014A000E8002E772093E80001C0B901FC0120E09C
:1014B0006115710579F1809196018823F1F18530EC
:1014C000F1F18091E80083FD3CC08091E80082FD4D
:1014D0002EC08091E80080FFEBCF2091F300809137
:1014E000F20090E0922B6115710551F08830910562
:1014F00038F421912093F100615071090196F3CFE6
:1015000021E0089709F020E08091E8008E77809331
:10151000E800CECF2111CFCF0AC080919601882359
:1015200061F0853061F08091E80083FD0AC0809110
:10153000E80082FFF2CF80E0089582E0089583E022
:10154000089581E008950895089580918B0108958C
:101550008093860170938801609387018091960142
:10156000843001F582E08093E9008FEF9091E800EC
:10157000815095FD06C095ED9A95F1F70000811117
:10158000F5CF8091E80085FF0DC040E050E063E0BA
:1015900070E086E891E00E94C5098091E8008E77AE
:1015A0008093E8000895BC0184E00C94A80ABC0173
:1015B00083E00C94A80ACF93DF9321E02093E90005
:1015C0002FEF3091E800215035FD06C035ED3A95FA
:1015D000F1F700002111F5CF2091E80025FF14C09C
:1015E000EC0140E050E068E070E00E94C5098091A5
:1015F000E8008E778093E80088E0FE01ACE8B1E077
:1016000001900D928A95E1F7DF91CF9108951F9394
:10161000CF93DF93CDB7DEB7AA970FB6F894DEBFAE
:101620000FBECDBFE8E9F1E080EA91E02091F10042
:1016300021938E179F07D1F780919901833009F488
:1016400061C030F4813071F0823009F49BC0B2C0C7
:101650008A3009F487C08B3009F46CC0893009F0F6
:10166000A9C020C080919801813A09F0A3C080915F
:10167000E800877F8093E80080919C0190919D0114
:10168000892B21F468E08CE891E003C060E080E001
:1016900090E070E00E94450A8091E8008B7780938B
:1016A000E80088C080919801813209F083C0809160
:1016B0009C0190919D01029708F07CC08091E80008
:1016C000877F8093E8008091E80082FD05C08091CB
:1016D00096018111F8CF6EC02091F3008091F20045
:1016E00090E0922B029731F48091F100813011F05B
:1016F000863021F48091F10080938B018091E80085
:101700008B7754C080919801813A09F053C0809141
:101710009C0190919D01892B09F04CC08091E800BB
:10172000877F8093E8008091E80080FFFCCF809164
:10173000000137C0809198018132E1F580919C01D0
:1017400090919D01892BB1F58091E800877F80936E
:10175000E8000E94F10980919A01809300010E94A3
:10176000E60228C080919801813221F58091E8003D
:10177000877F8093E8000E94F10980919B0180930C
:101780008A0118C080919801813AA1F48091E80003
:10179000877F8093E8008091E80080FFFCCF8091F4
:1017A0008A018093F1008091E8008E778093E800B1
:1017B0000E94F1098091E80083FFCEC180919801D9
:1017C00090919901492F50E04A30510508F0C4C169
:1017D000FA01EE59FF4F0C94C018803821F082387E
:1017E00009F0BAC108C080919401909195019923A4
:1017F00089F082600FC080919C018F70873008F063
:10180000ABC18093E9008091EB0085FB882780F9CC
:101810001092E9009091E800977F9093E800809300
:10182000F1001092F10065C1282F2D7F09F094C1BD
:10183000882319F0823061F08FC180919A01813044
:1018400009F08AC1933009F080E0809395012EC0A1
:1018500080919A0181112AC080919C018F702FEF95
:10186000280F263008F078C18093E9002091EB0022
:1018700020FF1CC0933021F48091EB00806214C0E3
:101880009091EB0090619093EB0021E030E0A90192
:1018900002C0440F551F8A95E2F74093EA00109268
:1018A000EA008091EB0088608093EB001092E900E1
:1018B0008091E800877F20C181114EC110919A016B
:1018C0001F778091E3008078812B8093E3008091E3
:1018D000E800877F8093E8000E94F1098091E8008A
:1018E00080FFFCCF8091E30080688093E3001111BA
:1018F00002C082E001C083E0809396012DC1805830
:10190000823008F029C180919A0190919B018C3D11
:1019100053E0950779F583E08A838AE289834FB79C
:10192000F894DE01139620E03EE051E2E32FF0E070
:1019300050935700E49120FF03C0E295EF703F5FA2
:10194000EF708E2F90E0EA3010F0C79601C0C0967D
:101950008D939D932F5F243149F74FBF8091E8000D
:10196000877F8093E8006AE270E0CE0101960E94D2
:10197000450AAEC040919C0150919D01292F33270B
:1019800023303105A9F068F42130310509F4F3C0A2
:101990002230310509F0E0C08BE390E0EAE4F1E0A9
:1019A00044C02132310521F12232310571F1D4C018
:1019B000992781309105A1F058F0029709F0CCC029
:1019C000E7E9F1E0E4918E2F90E0E7E9F1E02AC049
:1019D000EFECF1E0E4918E2F90E0EFECF1E022C02B
:1019E000EBEAF1E0E4918E2F90E0EBEAF1E01AC02F
:1019F0004115510509F4C4C04130510509F0ACC08E
:101A000089E090E0E5E7F1E010C04115510509F4E7
:101A1000BCC04130510509F09FC082E390E0E8ED81
:101A2000F0E003C0009709F497C02091E800277FF9
:101A30002093E80020919E0130919F018217930727
:101A400008F49C0140E02115310589F1809196014F
:101A5000882309F43DC08530D9F18091E80083FDE9
:101A600037C08091E80082FD2FC08091E80080FFA0
:101A7000EACF4091F3008091F20090E0942B211581
:101A8000310559F08830910540F444914093F100BC
:101A90003196215031090196F2CF41E0089709F0C3
:101AA00040E08091E8008E778093E800CCCF411130
:101AB000CDCF0AC080919601882351F0853041F046
:101AC0008091E80083FD04C08091E80082FFF2CF9E
:101AD0008091E8008B778093E8003EC08038E1F584
:101AE0008091E800877F8093E80080919701809340
:101AF000F1008091E8008E778093E8000E94F10960
:101B00002BC0811129C080919A0190919B01992746
:101B1000029714F58091E800877F8093E800109188
:101B20009A01109397010E94F109111106C080914A
:101B3000E30087FD02C081E001C084E0809396014C
:101B400042E061EC81E00E94100A42E261EC82E036
:101B50000E94100A809196018091E80083FF1AC0CC
:101B60008091E800877F8093E8008091EB0080629D
:101B70008093EB000FC082E190E0E5E8F1E055CF03
:101B800089E090E0ECE5F1E050CF80E490E0EAE01D
:101B9000F1E04BCFAA960FB6F894DEBF0FBECDBFD3
:101BA000DF91CF911F9108951F920F920FB60F9260
:101BB00011242F933F934F935F936F937F938F9352
:101BC0009F93AF93BF93CF93DF93EF93FF93C09116
:101BD000E900CF708091EC00D82FD17080FDD0E863
:101BE0001092E9008091F000877F8093F000789454
:101BF0000E94070B1092E9008091F00088608093AA
:101C0000F000CD2BCF70C093E900FF91EF91DF91F1
:101C1000CF91BF91AF919F918F917F916F915F9184
:101C20004F913F912F910F900FBE0F901F901895DD
:101C3000E8EDF0E080818E7F80831092E2001092C8
:101C4000DA001092E100A0EEB0E08C9181608C93FC
:101C500080818F77808319BCA7EDB0E08C918E7F57
:101C60008C9380818F7E8083109289010895CF921A
:101C7000DF92EF92FF920F931F93CF93DF93C8ED04
:101C8000D0E088818F7E8883E7EDF0E080818160FD
:101C9000808384E082BF81E08093890188818E7F88
:101CA000888302EE10E0F80110821092DA0081EED3
:101CB000C82ED12CF601108288818F778883888185
:101CC0008068888388818F7D888319BC10929601F3
:101CD00010929701109295011092940190EEE92EC6
:101CE000F12CF70180818B7F8083888181608883DC
:101CF00042E060E080E00E94100AF60180818E7F61
:101D00008083F80180818160808380818860808306
:101D1000F70180818E7F8083888180618883DF9155
:101D2000CF911F910F91FF90EF90DF90CF9008958A
:101D30001F920F920FB60F9211242F933F934F9340
:101D40005F936F937F938F939F93AF93BF93EF9323
:101D5000FF938091E10082FF09C08091E20082FF41
:101D600005C08091E1008B7F8093E1008091DA00D3
:101D700080FF2AC08091D80080FF26C08091DA00C1
:101D80008E7F8093DA008091D90080FF18C080E1B7
:101D900089BD82E189BD09B400FEFDCF81E0809359
:101DA00096018091890181110FC00E94180E0E9436
:101DB000370E8091E20084608093E20005C019BC78
:101DC00010929601109289018091E10080FF17C066
:101DD0008091E20080FF13C08091E2008E7F8093AB
:101DE000E2008091E20080618093E2008091D8005F
:101DF00080628093D80019BC85E080939601809121
:101E0000E10084FF30C08091E20084FF2CC080E1BB
:101E100089BD82E189BD09B400FEFDCF8091D80063
:101E20008F7D8093D8008091E1008F7E8093E100C8
:101E30008091E2008F7E8093E2008091E2008160D9
:101E40008093E20080919701882311F084E007C01D
:101E50008091E30087FD02C081E001C083E08093B0
:101E60009601809196018091E10083FF27C08091C7
:101E7000E20083FF23C08091E100877F8093E1002F
:101E800082E080939601109297018091E1008E7F0D
:101E90008093E1008091E2008E7F8093E200809148
:101EA000E20080618093E20042E060E080E00E9416
:101EB000100A8091F00088608093F000FF91EF910C
:101EC000BF91AF919F918F917F916F915F914F9152
:101ED0003F912F910F900FBE0F901F90189581E0AA
:101EE0008093E00080E28093D8001092C9008FE1D7
:101EF0009EE40197F1F700C0000087E090EBDC0161
:101F00008093230290932402A0932502B09326028B
:101F10009CE088E10FB6F894A895809360000FBE0E
:101F200090936000FFCF78941F920F920FB60F929C
:101F300011248F939F93AF93BF93809182019091CF
:101F40008301A0918401B09185010196A11DB11D6D
:101F50008093820190938301A0938401B0938501C3
:101F6000BF91AF919F918F910F900FBE0F901F90D7
:101F700018952FB7F8948091820190918301A091D8
:101F80008401B09185012FBF089580E0089590915C
:101F9000010292FF0DC0282F2871283019F4877F85
:101FA000846006C0282F2471243011F48B7F886050
:101FB00093FF0DC0282F2871283119F4877E846182
:101FC00006C0282F2471243111F48B7E8861209162
:101FD000020220FF0DC0382F3871383019F4877F86
:101FE000816006C0382F3171313011F48E7F8860E6
:101FF00021FF0DC0282F2871283119F4877E8161B7
:1020000006C0282F2171213111F48E7E886194FD44
:10201000877E0895F894E82FE295EF70F0E031A103
:10202000282F2F7081E090E001C0880F2A95EAF7F1
:10203000982F9095932391A392A1892B82A37894B2
:1020400008956F927F928F929F92AF92BF92CF929C
:10205000DF92EF92FF920F931F93CF93DF93CDB751
:10206000DEB72A970FB6F894DEBF0FBECDBFAE0124
:102070004F5F5F4F7A018AE0FA0111928A95E9F782
:102080000EE311E06A0166246394712C21E5822E2F
:1020900021E0922EF80180818F3F09F446C0F89428
:1020A000E82FE295EF70F0E021A18F70A30102C04C
:1020B000440F551F8A95E2F7CA01922F982B91A3DE
:1020C00092A18095892382A3789400C0E3E4F1E093
:1020D00021E030E0A12CB12C41914F3F89F0A42F99
:1020E000A295AF70B0E090968C9190E04F7002C0D6
:1020F000959587954A95E2F780FD02C0C90102C017
:1021000080E090E0A82AB92A220F331F8E169F067E
:1021100019F7F80180818F3F11F00E940A10F0EA50
:10212000FA95F1F7F601B182A0820F5F1F4FF2E03E
:10213000CF0ED11C41E00334140709F0ABCF4AE0C5
:1021400050E0B70183EF91E00E94C61811E00097BC
:1021500009F410E0892B89F08AE0F701A3EFB1E0E0
:1021600001900D928A95E1F781E08093F2010E943F
:10217000B90F9093F1018093F0018091F2018823CF
:10218000E9F12091F0013091F1014FB7F89480917D
:10219000820190918301A0918401B09185014FBF8C
:1021A000821B930B059750F18091F3019091F401FC
:1021B00090930402809303028091F5019091F601BF
:1021C00090930602809305028091F7019091F801A7
:1021D00090930802809307028091F9019091FA018F
:1021E00090930A02809309028091FB019091FC0177
:1021F00090930C0280930B021092F201812F2A9689
:102200000FB6F894DEBF0FBECDBFDF91CF911F9107
:102210000F91FF90EF90DF90CF90BF90AF909F9085
:102220008F907F906F900895CF93DF9382389105C0
:1022300069F1B0F48133910509F46FC048F4893233
:10224000910509F465C08A32910509F46BC08AC012
:102250008533910509F457C089339105B9F082C0DF
:10226000833E910571F138F4803E9105B1F0823ED4
:10227000910511F177C0863E9105B9F1873E910530
:10228000C9F1843E910509F06DC024C0209101027E
:1022900020FD53C021FD51C065C08091010280FD29
:1022A00046C08091020280FF48C08091010284FDF7
:1022B0003FC183EE90E03EC18091010282FF3AC0AF
:1022C000F4CF8091010282FD35C08091020280FD31
:1022D00034C0EBCF8091020281FF35C080910102B2
:1022E00084FD26C187EE90E025C18091010283FF25
:1022F00027C0F4CF8091010283FD22C080910202A9
:1023000081FD21C0EBCF8091010285FD1FC021C05E
:102310008091010285FD1DC019C08091010286FDDA
:102320001BC01DC08091010286FD19C015C089E344
:1023300090E000C182EE90E0FDC080EE90E0FAC037
:1023400086EE90E0F7C084EE90E0F4C089E290E081
:10235000F1C085E390E0EEC08AE290E0EBC081E35B
:1023600090E0E8C0811532E5930708F069C0811557
:1023700041E5940728F0982F8827816F906ADAC08A
:10238000883E910568F5803E910508F0D3C0883AF3
:102390009105B8F4853A910548F0855AE82FF0E0A8
:1023A000E35FFE4F808190E09064C4C0813091056E
:1023B00009F4BBC008F4BCC08430910508F4B8C06F
:1023C000B9C08F3B910508F0B3C0885AE82FF0E000
:1023D000EE0FFF1FE05FFE4F808191819464AAC0E1
:1023E000811520E59207F0F09C0174E03695279561
:1023F0007A95E1F7922F9370482F437021E030E0F7
:1024000002C0220F331F4A95E2F73C68392B8F70C8
:10241000982F9695969540E2949FC0011124822BA7
:10242000932B88C0811530E4930718F09F70906A51
:1024300081C09C013A9521153F4108F47BC078C0CA
:10244000EC01C11586E5D807E8F5C11525E5D207E9
:1024500048F08C2F0E94C70F8F7190E0982F88272B
:10246000906268C0C11534E5D30728F09C2F8827F7
:10247000846F906A5FC0AE01437055272C2F26955C
:102480002695C115D34578F481E090E002C0880F0D
:10249000991F4A95E2F740E2249F90011124822B74
:1024A000932B9C6847C081E090E002C0880F991F81
:1024B0004A95E2F740E2249F90011124822B932B4E
:1024C0009A6838C0C1152AE5D207F8F4C11539E574
:1024D000D30790F08C2F8F700E94C70F94E0D69591
:1024E000C7959A95E1F7CF70D0E0DC2FCC27D06963
:1024F0009E01282BC9011EC0C11548E5D407C0F0B4
:102500009C2F8827806F906A15C0CE019056811548
:10251000904270F48D2F8F710E94C70F282F2F715A
:10252000CE0199279062922B05C081E090E002C015
:1025300080E090E0DF91CF910895CF9384E090E028
:102540000E947E18C82F82E290E00E947E182C2FF5
:1025500030E0A901582BCA01CF91089569EE7EEFB2
:1025600080E090E00E94AA1860E082E090E00E9483
:102570008C1860E083E090E00E948C181092EC01CF
:102580001092ED011092EE011092EF0160E084E0F4
:1025900090E00E948C1860E082E290E00E948C182B
:1025A00060E085E090E00E948C1860E086E090E0BA
:1025B0000E948C186FEF87E090E00E948C1840E03A
:1025C00050E0BA0188E090E00E949E1860E08DE043
:1025D00090E00E948C1840E050E0BA0188E190E061
:1025E0000E949E1860E087E190E00E948C1840E015
:1025F00050E0BA018CE190E00E949E1860E070E02B
:1026000080E290E00E94AA1840E050E0BA0188E120
:1026100090E00E949E1840E050E0BA018FE090E008
:102620000E949E1840E050E0BA0183E190E00C94D3
:102630009E188091EB0181111092EB010895809515
:102640009091EA0189238093EA0108959091EA012B
:102650008091E901982B9093A0018091EB01882350
:1026600089F0892B8093A001E2EAF1E097E080E015
:10267000915029F021912223D9F38F5FF9CF811155
:102680000E94191348E050E061EE71E080EA91E0A9
:102690000E94C618892BA9F088E0E0EAF1E0A1EEDB
:1026A000B1E001900D928A95E1F7E0911E02F09160
:1026B0001F02309731F00280F381E02D80EA91E033
:1026C000099408952091E001809582238093E00190
:1026D000982F977099F430E0482F082E000C550B76
:1026E0002417350759F09091020292FD07C0859595
:1026F000859585950E9497021092E0010895CF93E9
:10270000C0910202C2FB992790F9981799F080FBBB
:10271000C2F9C09302026091010284E090E00E943D
:102720008C186C2F82E290E00E948C1882E0CF918E
:102730000C946213CF9108958091DF019091AE01C6
:10274000891719F08F5F8770FBCF08950F931F9340
:10275000CF93DF938091AD0182958F7009F05DC0BA
:102760008091AA01882309F458C08091DF0110915B
:10277000AE016091A8017091A901C091AB01D09107
:10278000AC0191E06F3F09F090E0292F06E081173E
:1027900009F443C0209721F07F3F21F030E003C0CF
:1027A00031E001C0322F90E030FD34C0089FF001CD
:1027B000099FF00D1124DF01A155BE4F11963C91E8
:1027C0001197371327C03C91361324C012963C91C1
:1027D000129731111FC013964D915C9114974C1BA9
:1027E0005D0B483C5105B0F48091AD018F70806164
:1027F0008093AD01EC54FE4F80818F7080618083A7
:1028000088EA91E00E943404DF91CF911F910F91EB
:102810000C949C1301968770BACFDF91CF911F91D2
:102820000F910895CF93DF93EC010E943E0226E4BE
:10283000829FC0011124FC012EE0D29FE00DF11D0A
:102840001124EC0FF11DEE0FFF1FED52FE4F85918D
:1028500094910E941411DF91CF9108959F92AF92AD
:10286000BF92CF92DF92EF92FF920F931F93CF937D
:10287000DF93CDB7DEB761970FB6F894DEBF0FBE1A
:10288000CDBF8C0185E0F801DE011D9601900D920F
:102890008A95E1F7F801E2809091A8016091A90181
:1028A0004091AB015091AC014115510531F06F3FA2
:1028B00031F481E09F3F19F403C081E001C080E062
:1028C000F82FF1709F2E80FD1AC1F801308121810F
:1028D000C380D48088EAA82E81E0B82EF090AA01A7
:1028E000F601E41BF50BFF2009F4C6C08091AD0191
:1028F000E83CF10508F091C0482F407F09F050C036
:10290000621311C093130FC0FE2CE1100CC08F7026
:1029100080618093AD01C5010E9434048091AD01B6
:10292000F801858329C1CD2831F02F3F31F481E0B2
:102930003F3F19F403C081E001C080E080FD03C087
:1029400081E08E2502C080E090E0F82FF170FF2E2C
:1029500080FF1CC08091DF014091AE0156E08417DA
:1029600009F4E8C090E0589FF001599FF00D112440
:10297000E155FE4F6181261306C06081631303C0D9
:102980006281E61203C001968770E9CFFE2CEE202B
:1029900009F4F2C08091AD0181608093AD0149C01E
:1029A000621306C0931304C0E11002C0F80186C090
:1029B000C8010E94C602882351F1EE2041F1209106
:1029C000AD01822F82958F7090E0029774F0809114
:1029D000A8019091A90198878F831986DB86CA8602
:1029E0002C87CE0107960E94340486E0F801A8EAFD
:1029F000B1E001900D928A95E1F70E94A6130AC0FA
:102A00006217C9F0C8010E94C60281111EC0C80128
:102A10000E943404FF24F394AFC0482F407F81F715
:102A200088EA91E00E94340486E0F50111928A95CB
:102A3000E9F7F12CA1C09313E5CFE110E3CFF80142
:102A40008583C8010E94340454C0EE2001F3209114
:102A5000AD01822F82958F7090E0029734F28091C1
:102A6000A8019091A9019A8389831B82DD82CC827F
:102A70002E83CE010196B7CFE83CF105D0F5FE2CB0
:102A8000EE2029F2621327C0931325C02091AD01D7
:102A900020FD18C0822F82958F70482F50E041157D
:102AA000510581F0F80125834F30510541F08F5FCA
:102AB000982F9295907F822F8F70892B8583C801E4
:102AC0000E94340486E0F801A8EAB1E001900D927A
:102AD0008A95E1F751C0C8010E94C602811185CFD5
:102AE0008091AD0181608093AD01C8010E943404E2
:102AF00043C086E0F50111928A95E9F73DC0EE20CA
:102B000009F485CFC8010E94C602F82E882309F473
:102B10007ECF86E0F801A8EAB1E001900D928A9597
:102B2000E1F78091A8019091A9010E9412140E94DE
:102B3000A61322C03D872E878D859E850E94121484
:102B4000292F22952F70223028F49F7039F081119F
:102B500005C00BC0243028F49F7049F4805E883093
:102B600020F0C8010E9434049F2CF92C05C0F80104
:102B70009581907F99F7F9CF8F2D61960FB6F894D4
:102B8000DEBF0FBECDBFDF91CF911F910F91FF90A0
:102B9000EF90DF90CF90BF90AF909F9008951F92DD
:102BA0000F920FB60F9211248F939F93AF93BF9301
:102BB00080912202811113C0809182019091830142
:102BC000A0918401B09185014196A11DB11D809312
:102BD000820190938301A0938401B0938501BF91FA
:102BE000AF919F918F910F900FBE0F901F901895EE
:102BF0009C01FC0132969FEF80E04191461789F0DD
:102C00009F3F19F4411101C0982F8F5F8630A9F7BB
:102C10009F3F39F0F901E90FF11D97FDFA956283A5
:102C20000895089520912002309121022817390734
:102C300071F09093210280932002E0911E02F091A6
:102C40001F02309721F00084F185E02D099408954A
:102C500020911C0230911D022817390771F09093C2
:102C60001D0280931C02E0911E02F0911F0230971A
:102C700021F00680F781E02D09940895E0911E026D
:102C8000F0911F02309721F00190F081E02D09941E
:102C900080E00895EF92FF920F93CF93DF93C42FBC
:102CA000D22FFC0182818823D1F040931B020E9425
:102CB000B90F90931A028093190280E28C0F88302A
:102CC00008F078C0C77081E001C0880FCA95EAF7A4
:102CD000DF91CF910F91FF90EF900C94F8028091CB
:102CE0001B02481356C02091190230911A024FB7A7
:102CF000F8948091820190918301A0918401B09118
:102D000085014FBF821B930B883C910508F041C0A1
:102D1000CD17C9F080E28C0F883040F4C77081E095
:102D200001C0880FCA95EAF70E94F10280E28D0F78
:102D3000883048F481E09D2F977001C0880F9A95E4
:102D4000EAF70E94F802093319F0E12CF12C03C0D4
:102D500080E5E82EF12C802F0E943303E114F1046A
:102D600051F08FE99FE00197F1F700C0000091E07A
:102D7000E91AF108F3CF802F0E94020380E28D0F41
:102D80008830C0F4D77081E001C0880FDA95EAF787
:102D90000AC080E28C0F883068F4C77081E001C0FF
:102DA000880FCA95EAF7DF91CF910F91FF90EF90CE
:102DB0000C94F102DF91CF910F91FF90EF90089565
:102DC000CF93DF93CDB7DEB72A970FB6F894DEBF67
:102DD0000FBECDBF84B7877F84BF0FB6F894A89588
:102DE00080916000886180936000109260000FBE47
:102DF00090E080E80FB6F8948093610090936100B2
:102E00000FBE85B7806885BF85B7806885BF85ECB4
:102E10009FE090935301809352010E94180E0E94EC
:102E2000370E8091E20084608093E2007894809174
:102E300096018823A1F01091E9001F709091EC0099
:102E4000892F817090FD80E8182B1092E900809105
:102E5000E80083FD0E94070B1F701093E90082E0D9
:102E600084BD93E095BD9AEF97BD80936E000EE30D
:102E700011E063E4E62E61E0F62ED8018D918D011C
:102E80008F3F11F00E940A10E016F106B1F703E43B
:102E900011E051E5E52E51E0F52EF80181918F0109
:102EA0008F3F11F00E940A10E016F106B1F78AE098
:102EB000E3E0F2E0DF01282F1D922A95E9F7E3EF26
:102EC000F1E0DF011D928A95E9F780E090E00E9431
:102ED0008618893E9E4F11F00E94AE1282E090E06B
:102EE0000E947E1880930D020E949D129093020210
:102EF000809301020E942110EFEFF6E721E0E150FC
:102F0000F0402040E1F700C000000E9421108091B5
:102F1000030280FF08C06FEF7FEF80E090E00E9427
:102F2000AA180E946F0F83E090E00E947E18682F1D
:102F300070E080E090E00E94BC0281E091E090931C
:102F40001F0280931E0230E4232E4DE0642E42E0E7
:102F5000742E80919601853009F043C012E1809172
:102F60009601853009F039C080919601843019F1BD
:102F70001092220288E190E00FB6F894A895809311
:102F800060000FBE2092600083B7817F846083BFA2
:102F900083B7816083BF7894889583B78E7F83BF22
:102FA0000FB6F894A89580916000886180936000C6
:102FB000109260000FBE80919501882309F4CFCF55
:102FC0000E942110E3E0F2E081919191892B09F0B8
:102FD0007EC06E167F06C1F7C2CF0E94E6020E9435
:102FE0003E160E942110882359F08FB7F894409123
:102FF00082015091830160918401709185018FBF9E
:1030000023E0A22E22E0B22E0EE012E0512C412C41
:10301000D5018D909D905D01F801C080D180C824BC
:10302000D924C114D10489F1312CEE24E394F12C7C
:10303000C6018E219F21892B11F139824A8221E01C
:10304000C4018E219F21892B09F420E02B830E944B
:10305000B90F8160782F9D838C8349815A816B8160
:103060008D810E948C03D8018D919C9111978E25A2
:103070009F258D939C935394BBE0B515F0F033944A
:10308000EE0CFF1CEEE03E12D3CF43940E5F1F4FB9
:10309000F5E04F12BDCF511010C08FEF8E838F839C
:1030A00018860E94B90F8160782F9A8789874E8190
:1030B0005F8168858A850E948C030E943E169091EC
:1030C0001802891709F445CF8093180242CF20E1F6
:1030D00029BD19BD09B400FEFDCF8091D8008F7DB8
:1030E0008093D8008091E00082608093E00080911E
:1030F000E00081FDFCCF0E94E60231CFF999FECFBE
:1031000092BD81BDF89A992780B50895A8E1B0E0F5
:1031100042E050E00C94B218262FF999FECF92BDF0
:1031200081BDF89A019700B4021639F01FBA20BD8C
:103130000FB6F894FA9AF99A0FBE08950396272FBE
:103140000E948D180E948C18252F0E948D18242F04
:103150000C948D180196272F0E948D180C948C18B2
:10316000DC01CB01FC01F999FECF06C0F2BDE1BD47
:10317000F89A319600B40D9241505040B8F7089536
:10318000EE0FFF1F0590F491E02D0994FB01DC0187
:1031900004C08D910190801921F441505040C8F72E
:0A31A000881B990B0895F894FFCFE7
:1031AA0001A50ADB0AA40AD70AD30AA30A818283E1
:1031BA00E200E900EA00B500B600B700CD008301DD
:1031CA00CC008A01920194012102230224022502E1
:1031DA00260227022A02B300B4006F0070003233BD
:1031EA00C69593F0F1F4F5F6F76766363594969737
:0231FA0034009F
:00000001FF
